:020000020000FC
:1000000013C04BC05AC00FC00EC00DC059C00BC0AA
:100010000AC009C008C007C006C005C004C003C0AC
:1000200002C001C000C0FFCF8FED8DBF2224442449
:1000300088245524662477242CBE20BE81E083BF0B
:1000400082E089BF8DE082BB82E781BB8DE285BF04
:1000500080EC8BBF28BA8FEF87BB789467FD02C016
:100060008895FCCF6F77862D8E7F49F0781629F022
:1000700010F4739401C0782E7CBE662021F494980D
:10008000969820BE09C083E280BF60FE03C09498AA
:10009000969A02C09698949AE1CF3FB6829B0BC085
:1000A000880C8099839481FA550C50F8441C47FEC3
:1000B000919847FC919A3FBE1895642C58BA1895B0
:0E00C0003FB673957F7309F460683FBE1895D4
:00000001FF
